:020000040000FA
:0400000069303A2801
:08000800A000030EA100831209
:100010008B1C32288B1031181428B11C3228643004
:10002000010203183128182800001628172818285C
:1000300019281A281B281C281D281E281F283110A3
:10004000B114A810031005190314AA0DA90DA80DC9
:10005000B00B322831152A08AF002908AE00280855
:10006000AD00B11081010B11210E8300A00E200EF6
:02007000090085
:0C007400203084008001840A6030040207
:10008000031C3C281230B0004A228316FF23900044
:10009000831283160C308505870183128501870141
:1000A000073099000030831691008312C830831600
:1000B0008100831231309000003083168C0083124F
:1000C00010308B00831600309B001C141A0883121A
:1000D000BC00851DCA233C1C7528831610309B006C
:1000E0001C141A088312BD002B23831620309B009A
:1000F0001C141A088312C1000130C1080319C10081
:1001000081018E018F010B118B100B108C018B174D
:1001100098203119AE202E22B30B96280310851992
:100120000314B90DF03039020319AF213C2388289C
:100130006400311808000B1D08000B11B1103114B8
:100140001230B000051DA928321483160113831242
:100150000800321083160117831208003111013094
:10016000B70085144008013ECE000F08CF008B1366
:100170002030370783169B001C141A088312A40032
:10018000A500C030A5061030370783169B001C144D
:100190001A088312A3000030370783169B001C1433
:1001A0001A088312A2008B17321CDC28220903399B
:1001B000A200A309A409A50922082D02031DA9294B
:1001C00023082E02031DA92924082F02031D4629F6
:1001D00001303702031DF3283C19F2283D18F3289B
:1001E0003D143E144B2202303702031DFE283C19F9
:1001F000FD28BD18FE28BD143E14582203303702D6
:10020000031D09293C1908293D1909293D153E14EA
:10021000652204303702031D14293C191329BD1926
:100220001429BD153E14722205303702031D1F2903
:100230003C191E293D1A1F293D163E147F22063007
:100240003702031D2A293C192929BD1A2A29BD165E
:100250003E148C2207303702031D35293C193429FE
:100260003D1B35293D173E14992208303702031DE6
:1002700040293C193F29BD1B4029BD173E14A62229
:1002800009303702031D46293E14B32225082F02E8
:10029000031DA92901303702031D55293C19542992
:1002A0003D1C55293D103E14DA2202303702031D51
:1002B00060293C195F29BD1C6029BD103E14DE2257
:1002C00003303702031D6B293C196A293D1D6B2938
:1002D0003D113E14E22204303702031D76293C19F9
:1002E0007529BD1D7629BD113E14E6220530370261
:1002F000031D81293C1980293D1E81293D123E1490
:10030000EA2206303702031D8C293C198B29BD1EB9
:100310008C29BD123E14EE2207303702031D9729A7
:100320003C1996293D1F97293D133E14F2220830AF
:100330003702031DA2293C19A129BD1FA229BD1303
:100340003E14F62209303702031DA8293E14FA2272
:10035000A929B70A0A30370203180800B728013064
:10036000B600B300B400B500B70085018701B11332
:100370009820B30BF529031085190314B90DF0303B
:10038000390203191C2AB41F8510B40BF52901305A
:1003900037020319FE220230370203190223033009
:1003A0003702031906230430370203190A230530E4
:1003B000370203190E2306303702031912230730C0
:1003C0003702031916230830370203191A2309309C
:1003D000370203191E233708B6080319B60003199C
:1003E000F3298514B6039630B400311DB8293111B4
:1003F000321CFF292D090339AD00AE09AF092F1CAE
:10040000B1132F1CB829B11BB8292E18B829B11760
:100410008B1320303707BB002F08BA00372210306B
:100420003707BB002E08BA00372200303707BB0061
:100430002D08BA0037228B17850187010830370253
:100440002030031985002A3003198700B70AB60146
:100450000A303702031CB8292B2308003E1C080071
:100460003E101030BB003D08BA00372208008B1345
:100470003A0883161C159A003B089B0055309D00D6
:10048000AA309D009C1464009C18432A1C118312FE
:100490008B17080008003C19871640083C1D4003D4
:1004A0004107D0000F08D100BC1925233D140800D6
:1004B0003C19071640083C1D40034107D2000F08B5
:1004C000D300BC192523BD1408003C19871540082A
:1004D0003C1D40034107D4000F08D500BC1925235B
:1004E0003D1508003C19051640083C1D4003410716
:1004F000D6000F08D700BC192523BD1508003C19EC
:10050000851640083C1D40034107D8000F08D9005C
:10051000BC1925233D1608003C19071540083C1D51
:1005200040034107DA000F08DB00BC192523BD1684
:1005300008003C19871440083C1D40034107DC00BB
:100540000F08DD00BC1925233D1708003C190714CE
:1005500040083C1D40034107DE000F08DF00BC19C6
:100560002523BD170800BC1908003C1DBB2A3030EC
:1005700085043F3087048E018F01C001D001D20174
:10058000D401D6010130D800DA00DC00DE004030B2
:10059000D1008030D300C030D500FF30D7004030CC
:1005A000D9008030DB00C030DD00FF30DF00FF30DD
:1005B000BD00080087128E018F01080007128E010E
:1005C0008F01080087118E018F01080005128E012E
:1005D0008F01080085128E018F01080007118E011E
:1005E0008F01080087108E018F01080007108E010F
:1005F0008F01080025238E018F0108000708203A8B
:10060000870008000708103A870008000708083A22
:10061000870008000508103A850008000508203A00
:10062000850008000708043A870008000708023A16
:10063000870008000708013A870008000508303ADB
:10064000850007083F3A87000800CF308505C03095
:100650008705BD0108003D188716BD1807163D190E
:100660008715BD1905163D1A8516BD1A07153D1BC0
:100670008714BD1B071408003C19402B3D1C4C2B54
:1006800050084002031D4C2B51080F02031C4C2B39
:100690003C1987123C1D87163C19502BBD1C5C2B46
:1006A00052084002031D5C2B53080F02031C5C2BF5
:1006B0003C1907123C1D07163C19602B3D1D6C2B85
:1006C00054084002031D6C2B55080F02031C6C2BB1
:1006D0003C1987113C1D87153C19702BBD1D7C2BC7
:1006E00056084002031D7C2B57080F02031C7C2B6D
:1006F0003C1905123C1D05163C19802B3D1E8C2B08
:1007000058084002031D8C2B59080F02031C8C2B28
:100710003C1985123C1D85163C19902BBD1E9C2B47
:100720005A084002031D9C2B5B080F02031C9C2BE4
:100730003C1907113C1D07153C19A02B3D1FAC2B84
:100740005C084002031DAC2B5D080F02031CAC2BA0
:100750003C1987103C1D87143C19B02BBD1FBC2BC6
:100760005E084002031DBC2B5F080F02031CBC2B5C
:100770003C1907103C1D07144E084002031DC52BF1
:100780004F080F02031CC52B85100C1C08000C1011
:10079000C00A0800B601B301B4013C1CD22BBC0155
:1007A000BC14DE2BBC1CD72BBC013C15DE2B3C1D26
:1007B000DC2BBC01BC15DE2BBC013C143C08B60094
:1007C0006400E22BE32BE42BE52BE62BB41B87160E
:1007D000B41F8712B30BE02BB40BE02B0310B60C45
:1007E000B608031DE02B0030BB003C08BA003722DE
:0207F0000800FF
:084000000800030003000200A8
:02400E00CC01E3
:10420000010003000300030003000200020002009B
:1042100002000000000000000000FF00FF00FF009F
:10422000000000000000000000000000000000008E
:104230000000C000C000C000C000FF00FF00FF0081
:104240000100C300F300CF00FF00C300F300CF0064
:10425000FF00C300F300CF00FF00FF00FF00FF00DE
:10426000FF00FF00FF00FF00FF00FF00FF00FF0056
:10427000FF00FF00FF00FF00FF00FF00FF00FF0046
:10428000FF00FF00FF00FF00FF00FF00FF00FF0036
:10429000FF00FF00FF00FF00FF00FF00FF00FF0026
:1042A000FF00FF00FF00FF00FF00FF00FF00FF0016
:1042B000FF00FF00FF00FF00FF00FF00FF00FF0006
:1042C000FF00FF00FF00FF00FF00FF00FF00FF00F6
:1042D000FF00FF00FF00FF00FF00FF00FF00FF00E6
:1042E000FF00FF00FF00FF00FF00FF00FF00FF00D6
:1042F000FF00FF00FF00FF00FF00FF00FF00AA001B
:00000001FF
